:020000040000FA
:1000000083160000073085000000003086000000E5
:100010008101000083128B0186010000B301B4014D
:10002000B501AC01B201CC20B10131085523B10AB0
:10003000FF3903191E28B72042231528CC200A3087
:10004000B10031085523B10AFF3903192A28B72016
:1000500042232128CC201D30B10031085523B10A9C
:10006000FF3903193628B72042232D28CC20A301BD
:10007000A401A50186018E20CC206E28051D5128E3
:10008000851C51282208A50721080318210FA40761
:1000900020080318200FA3072308FD218A108600DB
:1000A0003E284223051D5728851C65283E284923E4
:1000B000051D5728AC0A2C08243C031D6E28A301FB
:1000C000A401A5018E20AC0A6E284923851C652851
:1000D0002C08013C03183E28AC036E2883122C0820
:1000E000B20013233D30B7200310320D2C07B200AD
:1000F000FD208312A0000023B20A3208FD208312E3
:10010000A1000023B20A3208FD208312A2000023BE
:100110003D30B7202C08982083123E288312AC0172
:10012000B2010030A0000030A1002430A20008007D
:100130008312B1000310B10D310D6C3EB200B1015C
:100140003208FD208312B720B20AB10A3108033900
:100150000319AB28A0284830B7207A30B720CC202C
:1001600008008312D530AF00AF0BB428080083120B
:10017000AE000830AD008511B120AE0C0318C228C6
:100180008511C3288515B120AD0BBD288515B1207B
:10019000B120000000000800831230080D30B720A5
:1001A00000000A30B720B0000800B0010830AD00F0
:1001B0000518D8282623031005180314B00CAD0B1E
:0401C000DA28080031
:0601FA000A148A108207BE
:1002000000340034243400340034B5340034033472
:10021000893400340934573400340E342734003420
:1002200015343B3400341C344F3400342A347734D2
:10023000003438349F3400344634C73400345434E6
:10024000EF34003463341734003471343F340034F5
:100250007F34663400348D348E340034B034F2345C
:100260000034D43456340034F734B93401341B34F8
:100270001D3401343E34813401346134E4340134BA
:10028000853448340134A834AC340134CC341034CF
:100290000134EF34733402341234D7340234363438
:1002A0003B34023459349E3402347D3402340234F7
:1002B000A03466340234C334C9340234E7342D34F4
:1002C00003340A34913403342D34F5340334513477
:1002D000583403347434BC34203420342034313462
:1002E0002034203420343534203420343234353432
:1002F0002034203436343634203431343034303401
:1003000020343134353430342034323430343034E5
:1003100020343334303430342034343430343034D6
:1003200020343534303430342034363430343034C2
:1003300020343734303430342034383430343034AE
:100340002034393430343034313430343034303493
:10035000313432343534303431343534303430346F
:10036000313437343534303432343034303430345E
:10037000323432343534303432343534303430344D
:10038000323437343534303433343034303430343C
:10039000333432343534303433343534303430342B
:1003A000333437343534303434343034303430341A
:1003B0003434323435343034343435343034303409
:1003C00034343734353430343534303430343034F8
:1003D00035343234353430343534353430343034E7
:1003E00035343734353430343634303430343034D6
:0803F000363432343534303468
:0603FA008A140A108207BC
:1004000080347A3474346E34683462345C345634F4
:1004100050344A3445343F343A34353430342B3454
:10042000273422341E341A341734143410340E3462
:100430000B340934073405340434033402340234F1
:1004400001340234023403340434053407340934EB
:100450000B340E341034143417341A341E3422344E
:1004600027342B34303435343A343F3445344A342D
:10047000503456345C34623468346E3474347A34B4
:10048000803487348D34933499349F34A534AB341D
:10049000B134B734BC34C234C734CC34D134D6349C
:1004A000DA34DF34E334E734EA34ED34F134F3346E
:1004B000F634F834FA34FC34FD34FE34FF34FF34BF
:1004C000FF34FF34FF34FE34FD34FC34FA34F834A6
:1004D000F634F334F134ED34EA34E734E334DF3422
:1004E000DA34D634D134CC34C734C234BC34B73423
:1004F000B134AB34A5349F34993493348D3487347C
:1005000081347A3474346E34683462345C345634F2
:1005100050344A3445343F343A34353430342B3453
:10052000273422341E341A341734143410340E3461
:100530000B340934073405340434033402340234F0
:1005400001340234023403340434053407340934EA
:100550000B340E341034143417341A341E3422344D
:1005600027342B34303435343A343F3445344A342C
:10057000503456345C34623468346E3474347A34B3
:10058000803487348D34933499349F34A534AB341C
:10059000B134B734BC34C234C734CC34D134D6349B
:1005A000DA34DF34E334E734EA34ED34F134F3346D
:1005B000F634F834FA34FC34FD34FE34FF34FF34BE
:1005C000FF34FF34FF34FE34FD34FC34FA34F834A5
:1005D000F634F334F134ED34EA34E734E334DF3421
:1005E000DA34D634D134CC34C734C234BC34B73422
:1005F000B134AB34A5349F34993493348D3487347B
:100600008312B300330E0F39F63E0318073E3A3E0D
:10061000B72033080F39F63E0318073E3A3EB7209D
:100620002E30B72008008312B3003030B5000A30F6
:100630003302031C1E2BB300B50A172B30303307CF
:10064000B4003508B7203408B72008008312AA097F
:10065000AB09AB0A0319AA0AFA30A9003623A90B81
:100660002E2BAB0A0319AA0F2C2B0800372B382B83
:10067000392B3A2B3B2B3C2B3D2B3E2B3F2B402B3E
:100680000000080083120030AA003230AB0026239D
:10069000080083120030AA00FA30AB0026230800BD
:1006A0004923492349234923080083128900582BF1
:1006B000592B5A2B5B2B83165D2B5E2B0814602B5A
:0A06C0008312622B632B0808080068
:02400E00F23F7F
:10420000443444345334323435344D3468347A349D
:1042100020340034313436344634383434342D3498
:104220003034313433343034203447343834333458
:104230002D343234303420340034323435342F3499
:10424000303433342F343034363420344134443431
:104250003534383438340D340A345234533420343D
:10426000393436343034303462340D340A34003466
:00000001FF
